:020000040000FA
:100000008316851086100610061583128F019C0139
:100010009C14861006148510861402303E2086102B
:10002000103084000C308E00000006108001061D88
:1000300080140000840A0614000000008E0B1528AE
:100040000F3084000E308E000508FD3900040418BE
:10005000023A8500840A4E303E2000008E0B242890
:100060008510FF303E20FF303E20FF303E20FF3025
:100070003E2052303E20000064000C288C008C0B87
:040080003F2808000D
:02400E00FE3F73
:00000001FF
